S315080000009044002099020008A1020008A3020008F3
S31508000010A5020008A7020008A902000800000000BF
S31508000020000000000000000000000000AB0200080D
S31508000030AD02000800000000AF020008592D0008B4
S31508000040B3020008B3020008B3020008B3020008AE
S31508000050B3020008B3020008B3020008B30200089E
S31508000060B3020008B3020008B3020008B30200088E
S31508000070B3020008B3020008B3020008B30200087E
S31508000080B3020008B3020008B3020008B30200086E
S31508000090B3020008B3020008B3020008B30200085E
S315080000A0B3020008B3020008B3020008B30200084E
S315080000B0B3020008B3020008B3020008B30200083E
S315080000C0B3020008B3020008B3020008B30200082E
S315080000D0B3020008B3020008B3020008B30200081E
S315080000E0B3020008B3020008B3020008B30200080E
S315080000F0B3020008B3020008B3020008B3020008FE
S31508000100B3020008B3020008B3020008B3020008ED
S31508000110B3020008B3020008B3020008B3020008DD
S31508000120B3020008B3020008B3020008B3020008CD
S31508000130B3020008B3020008B3020008B3020008BD
S31508000140B3020008B3020008B3020008B3020008AD
S31508000150B3020008B3020008B3020008B30200089D
S31508000160B3020008B3020008B3020008B30200088D
S31508000170B3020008B3020008B3020008000000003A
S31508000180B3020008B3020008B3020008B30200086D
S31508000190B3020008B3020008B3020008B30200085D
S315080001A0B3020008B3020008B3020008B30200084D
S315080001B0B3020008B3020008B3020008B30200083D
S315080001C0B3020008B302000800000000B3020008EA
S315080001D0B3020008B3020008B3020008B30200081D
S315080001E0B3020008B3020008B3020008B30200080D
S315080001F0B3020008B302000800F002F800F03CF869
S315080002000AA090E8000C82448344AAF10107DA4563
S3150800021001D100F031F8AFF2090EBAE80F0013F079
S31508000220010F18BFFB1A43F001031847D447000013
S31508000230F4470000103A24BF78C878C1FAD85207A4
S3150800024024BF30C830C144BF04680C607047000042
S315080002500023002400250026103A28BF78C1FBD8C1
S31508000260520728BF30C148BF0B6070471FB504F05E
S3150800027067FB1FBD10B510BD00F09CF91146FFF7CE
S31508000280F5FF03F088FA00F0BAF903B4FFF7F2FFB6
S3150800029003BC00F0C1F90000094880470948004737
S315080002A0FEE7FEE7FEE7FEE7FEE7FEE7FEE7FEE718
S315080002B0FEE7FEE704480549054A064B7047000075
S315080002C0052E0008F9010008903E00209044002001
S315080002D0904000209040002053EA020C00F069800C
S315080002E02DE9F04B4FF00006002B1FBFB3FA83F53C
S315080002F003FA05F424FA05F65E4012BF1643B2FA6D
S3150800030082F502FA05F4C5F120051EBF22FA05FC9E
S3150800031044EA0C04203556EA044C4FEA144418BF44
S31508000320641C4FF000084FF00009904271EB030C73
S3150800033039D3002919BFB1FA81F701FA07F6B0FADD
S3150800034080F700FA07F6C7F120071EBF20FA07FC58
S3150800035046EA0C062037B6FBF4FCA7EB0507103F68
S3150800036007F01F0BCBF120060CFA0BFB2CFA06F64E
S3150800037044BFB3460026202FA4BF5E464FF0000BAD
S315080003805BEA060C08BF4FF0010B19EB0B09ABFB38
S31508000390027C48EB0608C01B06FB02CC0BFB03CC11
S315080003A071EB0C01C1E70B46024641464846BDE8DB
S315080003B0F08B13B54FF000004FF00001AFF300804B
S315080003C0BDE81C40704740EA010310B59B070FD1F2
S315080003D0042A0DD310C808C9121F9C42F8D020BAA7
S315080003E019BA884201D9012010BD4FF0FF3010BD5F
S315080003F01AB1D30703D0521C07E0002010BD10F82D
S31508000400013B11F8014B1B1B07D110F8013B11F8F2
S31508000410014B1B1B01D1921EF1D1184610BD032AB0
S3150800042040F2308010F0030C00F0158011F8013B03
S31508000430BCF1020F624498BF11F801CB00F8013BEA
S3150800044038BF11F8013BA2F1040298BF00F801CBAE
S3150800045038BF00F8013B11F0030300F05280083A58
S31508000460C0F0088051F8043B083A51F804CBA0E8DC
S315080004700810F5E7121D5CBF51F8043B40F8043B31
S31508000480AFF30080D20724BF11F8013B11F801CB66
S3150800049048BF11F8012B24BF00F8013B00F801CB37
S315080004A048BF00F8012B704702F0FF0343EA032216
S315080004B042EA024200F002B84FF000020429C0F0F6
S315080004C0128010F0030C00F05080CCF1040CBCF143
S315080004D0020F18BF00F8012BA8BF20F8022BA1EBCA
S315080004E00C0100F042B85FEAC17C24BF00F8012B7A
S315080004F000F8012B48BF00F8012B7047704770477A
S31508000500704710B5203AC0F00B80B1E81850203A71
S31508000510A0E81850B1E81850A0E81850BFF4F5AF95
S315080005205FEA027C24BFB1E81850A0E8185044BF1F
S3150800053018C918C0BDE810405FEA827C24BF51F88C
S31508000540043B40F8043B08BF7047D20728BF31F880
S31508000550023B48BF11F8012B28BF20F8023B48BFD1
S3150800056000F8012B70474FF0000200B51346944679
S315080005709646203922BFA0E80C50A0E80C50B1F1ED
S315080005802001BFF4F7AF090728BFA0E80C5048BF01
S315080005900CC05DF804EB890028BF40F8042B08BF9F
S315080005A0704748BF20F8022B11F0804F18BF00F89B
S315080005B0012B7047754600F02BF8AE4605006946D4
S315080005C0534620F00700854618B020B5FFF772FE9F
S315080005D0BDE820404FF000064FF000074FF0000836
S315080005E04FF0000B21F00701AC46ACE8C009ACE8B7
S315080005F0C009ACE8C009ACE8C0098D46704710B51B
S315080006000446AFF300802046BDE81040FFF73DBE24
S3150800061000487047303E002001491820ABBEFEE76F
S3150800062026000200704700F0E8F8FCE710B500F075
S315080006309DF8012812D00A4C207801280ED102F024
S315080006400BFCD4E90112114401F5FA71884205D36D
S3150800065000202070BDE8104000F0E8B810BD00008A
S3150800066060000020014840687047000060000020D4
S3150800067010B504490120087000F006F8BDE81040DE
S31508000680FFF7D4BF6000002010B5044C207801287D
S3150800069002D102F0E1FBA06010BD0000600000205E
S315080006A001494860704700006000002010B500F05E
S315080006B0A8F800F09DF802F0D7FB02F079FA00F0EE
S315080006C049F8BDE81040FFF7D3BF10B500F095F81C
S315080006D002F0E2FB00F052F8BDE81040FFF7A6BFB3
S315080006E010B502F043F9034903200870BDE810402D
S315080006F0FFF7CABF6C000020704700000948007861
S31508000700002807D0012807D0022807D0032807D0D9
S3150800071040207047402070470020704700207047EF
S31508000720402070476C00002009480078002807D050
S31508000730012807D0022807D0032807D04020704791
S3150800074040207047002070470020704740207047BF
S315080007506C00002010B502F0ABFD02F0A9FB0249BF
S315080007600020087010BD00006C00002010B50024A1
S3150800077002F0ACFD00B10124204610BD38B50E4884
S31508000780694602F0BDFB0D4C012806D100202070F9
S315080007909DF80010084802F0A3FD0748694602F0D4
S315080007A037F9012806D1032020709DF80010024869
S315080007B002F096FD38BD0000D83100206C000020FC
S315080007C070B506460C46094D2878002803D13046F0
S315080007D0E1B202F0EBFB2878032803D13046E1B2F8
S315080007E002F0B6F9BDE8704002F0E6BD6C000020E4
S315080007F0AFF30080642002F02FB8AFF3008002F058
S3150800080031B8AFF3008072B6704762B6704770B5FC
S3150800081005460C46164605E014F8010B05F8010BCB
S31508000820FFF7EBFF761EB6B2F6D270BD10B502F032
S31508000830C1F9C0B100F024F8C8B1FFF75DFF02F0B6
S3150800084025FB00F0F7FB02F0B1F90B4908400B490C
S31508000850086002F0ABF94468FFF7D7FFA047BDE888
S315080008601040FFF73DBFBDE81040FFF739BFBDE8B0
S315080008701040FFF735BF000080FFFF1F08ED00E0BE
S3150800088010B506484FF4005101F098F9012803D035
S3150800089001F0DAFF012010BD002010BD000802405B
S315080008A0006800F58050816941F002018161704756
S315080008B0006800F58050816941F4005181617047F4
S315080008C038B50446206800F58050816941F48011E6
S315080008D08161206800F5805080690090012000F051
S315080008E0C3FB2068009900F58050816138BD00007F
S315080008F05379107940EA0323074808440364D378F8
S31508000900117841EA0361937852781B0443EA02227C
S315080009101143416470470000008002402DE9F04110
S31508000920AEB00446002904D04FF40060E060C00071
S31508000930A060002511951295139514951595169591
S31508000940E06900287DD017954FF400701890199526
S315080009501A951B951C951D9540271E971F95209542
S3150800096021952295239524952595269580262796C3
S31508000970289529952A952B952C952D9520680268FA
S3150800098045490A40D4E902131943179B194341F410
S315080009900071114301602068D0F80080012000F042
S315080009A063FB2068C0F800802068476020684768B5
S315080009B0012000F059FB20684760206885602068A0
S315080009C0C560206881694FF64172114041F0800187
S315080009D0816120688769012000F046FB20688761ED
S315080009E02068C5612068C769012000F03DFB2068C2
S315080009F0C7610195B004029003950111049105950C
S31508000A00069507950895042109910A9040120B90BE
S31508000A1080010C9040120D900E960F951095206847
S31508000A2000F5805081691D4A11401D4A0A438261BA
S31508000A30206800F580508569012000F015FB2068C4
S31508000A4000E016E000F5805085612068154900F53C
S31508000A5080500160206800F580500568012000F08C
S31508000A6003FB206800F580500560A069012804D0C2
S31508000A700AE04FF48060179066E7206800F580501A
S31508000A80C169094A1143C16162692EB02046002135
S31508000A90BDE8F041FFF72CBF0F8120FF233FDEF8AA
S31508000AA0040020028020C1024000010038B5044637
S31508000AB02068016841F00401016020680068009020
S31508000AC0012000F0D1FA21680098086038BD38B5D1
S31508000AD004462068016841F0080101602068006842
S31508000AE00090012000F0C0FA21680098086038BD1F
S31508000AF00022002905D001291FD0022920D04FF451
S31508000B0040720B2800D9001D0F490B6823F4407367
S31508000B100B600B6813430B600A6822F0F8020A6040
S31508000B200A68022303EBC00002430A60086840F41F
S31508000B3080300860BFF34F8F70474FF48072E0E74C
S31508000B404FF40072DDE70000103C0240104A1368BB
S31508000B5023F44073136003290FD0022913D01168B8
S31508000B6041F00401116011684FF4803343EA002014
S31508000B7001431160BFF34F8F7047116848F20403B1
S31508000B8019431160EFE7116841F400411160EAE783
S31508000B90103C0240074A136823F440731360136835
S31508000BA01360136843F0010313600170BFF34F8F9E
S31508000BB070470000103C024010B509490C6824F43F
S31508000BC040740C600C6844F440740C600C6844F083
S31508000BD001040C6002604360BFF34F8F10BD000034
S31508000BE0103C0240084A136823F4407313601368E4
S31508000BF043F480731360136843F0010313600180A4
S31508000C00BFF34F8F70470000103C0240084A136834
S31508000C1023F440731360136843F400731360136876
S31508000C2043F0010313600160BFF34F8F7047000064
S31508000C30103C0240134908688207134803D58269A5
S31508000C4042F0200282610A68D20603D5826942F020
S31508000C50100282610A68920603D5826942F0080288
S31508000C6082610A68520603D5826942F004028261EB
S31508000C700A68120603D5826942F002028261F220EE
S31508000C80086070470C3C0240D400002070B504464A
S31508000C9011490020886100F09FFF05460F4E09E0C4
S31508000CA0601C07D024B100F097FF401BA04201D971
S31508000CB0032070BD3068C003F2D4306810F0F20F1C
S31508000CC003D0FFF7B7FF012070BD3068C00701D019
S31508000CD001203060002070BDD40000200C3C02408A
S31508000CE02DE9F04704460D4616461F464FEA552994
S31508000CF04FEA49292068401C04D14946204600F09D
S31508000D00C9F838B32068484505D04946204600F05A
S31508000D10D3F8044604B32068281A05192D1D4FF484
S31508000D20007809F50079FFF768FD281B001F404584
S31508000D3006D34946204600F0BFF8044674B1251D7F
S31508000D4016F8010B05F8010B7F1E002FEBD10120C9
S31508000D50BDE8F0870020FBE70020F9E70020F7E769
S31508000D6010B50B480068401C03D0094800F016F976
S31508000D7048B108480068401C03D0064800F00EF940
S31508000D8018B1012010BD002010BD002010BD0000C4
S31508000D90683400206432002070B505460C460D48BC
S31508000DA0411B601E814201D2002070BD284600F01A
S31508000DB03FF806462819401E00F03AF80146FF2E6D
S31508000DC006D0FF2904D03046BDE8704000F004B8CC
S31508000DD0002070BDFFFF1F0870B586B004460E469A
S31508000DE0012500200090B44200D900250CB10B2E35
S31508000DF000D90025012D17D1019002200590012068
S31508000E00049000F027FD0BE0FFF7F7FC039401A818
S31508000E10694600F089FC08B1002503E0641CE4B2C9
S31508000E20B442F1D900F0CAFC06B0284670BD0000ED
S31508000E302DE9F0410546FF2700240E4EFFF7DDFC9D
S31508000E4004EB440156F82120AA420BD806EB810090
S31508000E5040681044A84205D904EB440006EB80001C
S31508000E60077A03E0641CE4B20B2CE7D33846BDE8E6
S31508000E70F08100006C4900080048704700800008AF
S31508000E8003494FF0FF30086001F5017108607047AB
S31508000E906432002010B5CA0501D0002010BD0268D2
S31508000EA08A4201D1012010BD02C04FF40072FFF73B
S31508000EB0AEFC012010BD000070B504460D460D4875
S31508000EC0844202D1A0F5017409E00B48854202D19B
S31508000ED0084C054603E0204600F060F830B1294684
S31508000EE02046FFF7D7FF18B1204670BD002070BD19
S31508000EF0002070BD68340020008000080B48016897
S31508000F004268114482681144C26811440269114456
S31508000F104269114482691144D0F8F801084400284E
S31508000F2001D00020704701207047000000800008AB
S31508000F3070B504460D4616461448011B681E8142C4
S31508000F4001D2002070BD2046FFF772FFFF2812D09D
S31508000F506019401EFFF76CFFFF280CD0600A40029C
S31508000F600B49884209D12B46324621460948BDE835
S31508000F707040FFF7B5BE002070BD2B4632462146AD
S31508000F800548BDE87040FFF7ABBE0000FFFF1F082D
S31508000F900080000868340020643200202DE9F04102
S31508000FA006464FF0010800F055FC0024306800EBB7
S31508000FB0840706EB84004568FFF71FFC00232A46D2
S31508000FC00220394600F004FC10B14FF0000808E092
S31508000FD03868A84202D04FF0000802E0641C802C52
S31508000FE0E4D300F0EBFB4046BDE8F08108B50020ED
S31508000FF000900E480168491C15D041688268114462
S31508001000C268114402691144426911448269114453
S31508001010C0690844C043401C0090054804216A463C
S31508001020FFF786FF08BD012008BD000068340020D0
S31508001030F881000810B50B4A4FF0FF301060002108
S315080010401160121D10601160064A103A1060116096
S31508001050121D10601160121D1060116000F0ECFD89
S31508001060002010BD2038024070B5044600F0B4FDDB
S315080010700546601C02D004480078044400F0ACFD24
S31508001080401BA042FAD370BD40000020F0B50024F2
S3150800109090F84550012D09D0012780F845700225A2
S315080010A080F84450816244F2F45C19E00220F0BDF5
S315080010B001EB44154FF000462E60C5F804C0C4EB9A
S315080010C0C41606EB460602EB8606AE6086695E1E09
S315080010D0B44203D205F12006EE6000E0E960641C24
S315080010E09C42E5D3026802F58052D16080F84470CC
S315080010F0002180F845100020F0BD2DE9F0430025B9
S3150800110090F84540012C0BD04FF0010C80F845C0F3
S31508001110022480F84440C1625F1E4FF480181CE028
S315080011200220BDE8F08301EB4514C4F80080C5EB46
S31508001130C51606EB460602EB8606A660C66926B9FC
S31508001140266846F44009C4F80090BD4203D204F16B
S315080011502006E66000E0E1606D1C9D42E3D302686C
S3150800116002F58052116180F844C0002180F84510CC
S315080011700020D6E710B590F84510012913D00123B1
S3150800118080F84530022180F84410816A0A680024F4
S31508001190002A29DB0A68D20518D5826B521C82639D
S315080011A0012A02D002E0022010BD01632830C16086
S315080011B00A68C2F30D42121F426182689268826110
S315080011C0C968016003774477002010BD0A68920554
S315080011D005D5016344638363C968816204E0826B51
S315080011E0521C8263C968816200F8443F447001203A
S315080011F010BD00002DE9FC47044600260196B046BE
S31508001200002C03D094F8440018B107E00120BDE88B
S31508001210FC8784F84560204600F002F976480168A4
S3150800122041F480410160006800F4804000907348F2
S31508001230016821F4000101600168226A1143016016
S31508001240206800F58050016841F00101016000F056
S31508001250C3FC05464FF4FA7709E000F0BDFC401BD5
S31508001260B84204D9032004F8440F6670CFE7206813
S3150800127000F580500068C007EFD12068006920F0AB
S315080012801C0500F0A9FE5E495E4A0144914202D25D
S3150800129045F0080516E05C495C4A0144914202D2D1
S315080012A045F00C050EE05A495A4A0144914209D3C1
S315080012B0594908445949884202D245F0040501E0D3
S315080012C045F010052068056100214FF400422046CC
S315080012D000F0ECF9012538B101212046FFF71EFB85
S315080012E084F84450012092E7FF20FFF7BDFE6068AE
S315080012F0F0B300F071FC074641F288390121204617
S3150800130001AA00F0E7F800F067FCC01B484508D9B9
S3150800131001212046FFF702FB04F8445F66700320AC
S3150800132075E701984007E9D5002120464FF4805219
S3150800133000F0BCF938B101212046FFF7EFFA84F82E
S315080013404450012063E700F047FC07462046012188
S3150800135001AA00F0BFF800F03FFCC01B48450AD9B7
S3150800136001212046FFF7DAFA04F8445F667000E0C8
S3150800137022E003204BE701988006E7D51021204696
S3150800138001AA00F0A7F838B101212046FFF7C6FAEE
S3150800139084F8445001203AE70198410703D54FF4F1
S315080013A00061E16000E0E660800701D5A6601BE009
S315080013B04FF48040A06017E0E0680021C0F3CF0238
S315080013C0A068C0F34F000243204600F06FF938B119
S315080013D001212046FFF7A2FA84F84450012016E7B7
S315080013E040F6FF70FFF740FE41462046FFF796FAA3
S315080013F084F8445000200AE7443802400438014083
S3150800140000D3CEFEC0E1E40040F1E9FD40787D015D
S3150800141000796CFC005A6202001F0AFA80F0FA0290
S31508001420F0B587B000682549884245D12448016847
S3150800143041F000710160016801F0007101910168D5
S3150800144041F080610160016801F0806101910168E5
S3150800145041F000610160006800F0006001903220F0
S3150800146002900224039400250495032605960B276B
S315080014700697144802A900F0B1FA86200290039450
S3150800148004950596069702A90F4800F0A7FA2003C7
S315080014900290039404950596069702A90B4800F056
S315080014A09DFA4FF4205002900394049505960697EA
S315080014B002A9074800F092FA07B0F0BD0080024082
S315080014C03038024000080240000002400004024092
S315080014D0001802402DE9F0470446914694F8440066
S315080014E082281DD0822084F844002068026902F010
S315080014F01C03228A4FF6FF7505EAC2221A434FF4E7
S31508001500F86303EA8111114321F0020141F0010554
S31508001510056100F061FB064601274FF480380FE0AD
S315080015200220BDE8F08700F057FB801B404505D335
S3150800153004F8447F002060700320F2E720680569FC
S31508001540E807F0D12068406980B2C9F8000084F83D
S3150800155044700020E5E770B5044694F84500012874
S3150800156019D0012584F84550022084F84400204605
S31508001570FFF7ADFA2046FFF799FA2046FFF7A0F9DC
S315080015802046FFF795F92046FFF78AF904F8445FE5
S315080015900020607070BD022070BDF0B5002390F881
S315080015A04520012A11D0012780F84570022280F8CB
S315080015B04420002659B1C46A2268002A0CDA12218E
S315080015C000F8441F46700120F0BD0220F0BD00F867
S315080015D0447F46700120F0BD40F2F455A9420AD96D
S315080015E0B1FBF5F2B1FBF5FC05FB1C1CBCF1000FC9
S315080015F002D0521C00E00122012A44D1226842F09E
S3150800160040522260C26AC1F30C015160C16A0A687D
S3150800161042F000420A60C16AC968C16235E0C46A1C
S31508001620D4F800C02CF0405CC4F800C033B9C46AD2
S31508001630D4F800C04CF0805CC4F800C0C46A656089
S31508001640541EA34214D1C46AD4F800C04CF0005CFE
S31508001650C4F800C0C2F10104C4EBC41404EB44048A
S3150800166001EB8404D0F82CC0C4F30C04CCF8044075
S31508001670C46AD4F800C04CF0004CC4F800C0C46A70
S31508001680E468C4625B1C9342C9D3016801F58051C2
S315080016904A69520705D504224A61016801F5805155
S315080016A04E6000F8447F46700020F0BD2DE9F041F9
S315080016B0044694F84400422820D0422084F8440086
S315080016C02068036903F01C03258A4FF6FF7606EAAD
S315080016D0C5251D434FF4F86303EA8111294341F0F8
S315080016E0020141F0010591B241612068056100F0EF
S315080016F073FA064601274FF480380FE00220BDE84A
S31508001700F08100F069FA801B404505D304F8447F50
S31508001710002060700320F2E720680569E807F0D129
S3150800172084F84470EBE700002DE9F04704460E46BE
S31508001730DFF8808098F81400012809D0012088F87D
S3150800174014004CF250394846FFF7A0FA18B12CE0BD
S315080017500220BDE8F0874FF0FF3131602168164F4F
S31508001760012901D0A5681BE0207C6168FFF7EEF926
S315080017704846FFF78BFA396848F204029143396004
S3150800178013E0217C2846FFF7B3F94846FFF77EFAAF
S31508001790396821F0FA01396008B1356005E06D1C39
S315080017A0D4E902211144A942EBD8002188F8141083
S315080017B0CFE70000D4000020103C0240034801682F
S315080017C041F000410160002070470000103C0240D3
S315080017D02DE9F0470646894614461D461B4F387DB7
S315080017E0012808D0012038754CF250384046FFF7DA
S315080017F04DFA18B126E00220BDE8F08736B1012E71
S3150800180009D0022E0CD0032E14D10EE04846E1B2C0
S31508001810FFF7C0F90EE0A1B24846FFF7E3F909E081
S3150800182021464846FFF7F2F904E022462B46484689
S31508001830FFF7C2F94046FFF729FA05490A6822F078
S3150800184001020A6000213975D6E70000D40000209D
S31508001850103C0240002007490A68002A09DA054AAE
S31508001860054B0C3A1360054B13600968002900DA2A
S3150800187001207047103C024023016745AB89EFCD34
S315080018802DE9F04F0023DFF824810F274FF0010CD4
S315080018900CFA03F201EA020494427DD10668032594
S315080018A04FEA430905FA09F5AE430660DE0800EB80
S315080018B08609D9F820A05E074FEAD66B3E4607FA96
S315080018C00BFB2AEA0B0AC9F820A0D0F8089029EAE7
S315080018D00509C0F80890D0F8049029EA0209C0F86A
S315080018E00490C268AA43C26023F0030202EB08050B
S315080018F0D5F808284FEA83794FEA197906FA09F6DE
S3150800190006EA020A2A4A904201D100222DE0294A13
S31508001910904201D1012228E0274A904201D10222B1
S3150800192023E0264A904201D103221EE0244A90422F
S3150800193001D1042219E0234A904201D1052214E07C
S31508001940214A904201D106220FE0204A904201D155
S3150800195007220AE01E4A904201D1082205E01D4AE4
S31508001960904201D1092200E00A2202FA09F2524500
S3150800197016D1D5F80828B243C5F80828164A1568B6
S31508001980A5431560121D1568A5431560121D156837
S31508001990A5431560121D00E002E01568A543156011
S315080019A05B1C102BFFF474AFBDE8F08F00300140CC
S315080019B0000002400004024000080240000C0240F9
S315080019C0001002400014024000180240001C0240A9
S315080019D00020024000240240003C01402DE9F84F57
S315080019E00022DFF8A491DFF8A0814FF0010E09F17B
S315080019F008094FF00F0C09F1040A0EFA02F60B68F3
S31508001A003340B34271D14C68022C01D0122C11D14B
S31508001A10D40800EB84073D6A5407E40E0CFA04FB6D
S31508001A2025EA0B05D1F810B00BFA04FB4BEA050BB7
S31508001A30C7F820B0076854000325A540AF4391F8BE
S31508001A4004B00BF0030B0BFA04FB4BEA070BC0F8C8
S31508001A5000B04F68012F05D0022F03D0112F01D0F7
S31508001A60122F11D18768AF43D1F80CB00BFA04FBDB
S31508001A704BEA070BC0F808B04768B7430E79C6F3B8
S31508001A80001696403E434660C668AE438D68A5403C
S31508001A903543C5604C68E4006FD53C4C256845F471
S31508001AA080452560246804F480440094384C22F06C
S31508001AB003052544D5F808789407260F0CFA06F48A
S31508001AC0A743344CA04201D100242EE0324CA04258
S31508001AD001D1012429E0314CA04201D1022424E09D
S31508001AE02F4CA04202D103241FE046E02D4CA04211
S31508001AF001D1042419E02C4CA04201D1052414E09C
S31508001B002A4CA04201D106240FE0294CA04201D15B
S31508001B1007240AE0274CA04201D1082405E0264CF8
S31508001B20A04201D1092400E00A24B4403C43C5F888
S31508001B300848D8F800409C434D68ED0300D51C437F
S31508001B40C8F80040104D2D1D2C689C434E68B603FE
S31508001B5000D51C432C60D9F800409C434D68ED0223
S31508001B6000D51C43C9F80040DAF800409C434D688C
S31508001B70AD0200D51C43CAF80040521C102AFFF4D7
S31508001B803CAFBDE8F88F0000003C014044380240F5
S31508001B9000300140000002400004024000080240F4
S31508001BA0000C0240001002400014024000180240D7
S31508001BB0001C02400020024000240240006908423E
S31508001BC001D00120704700207047002A01D08161AA
S31508001BD0704709048161704701F03EB910B50320CA
S31508001BE000F008F9002000F005F800F06BF8002076
S31508001BF010BD000070B504460D4D4FF47A71287873
S31508001C00B1FBF0F00B490968B1FBF0F000F00CFCF1
S31508001C1008B1012070BD102C07D200222146501EA3
S31508001C2000F0C8F86C60002070BD012070BD00008F
S31508001C30400000205400002010B51E4C00228021D0
S31508001C402046FFF7C2FF80212046FFF719FE1A48F3
S31508001C504FF40051FFF714FEA115184C2046FFF764
S31508001C600FFE61152046FFF70BFE1549086820F49C
S31508001C708020086012481038026822F0400202608C
S31508001C80026822F008020260026822F0040202607A
S31508001C90026822F002020260026822F00102026073
S31508001CA0086820F080500860081D016821F480410A
S31508001CB0016010BD0004024000080240000C02400A
S31508001CC04038024030B587B03649086840F0805041
S31508001CD00860086800F080500190081D026842F408
S31508001CE080420260006800F4804001902D48103858
S31508001CF0026842F001020260026802F001020192E3
S31508001D00026842F002020260026802F002020192D0
S31508001D10026842F004020260026802F004020192BC
S31508001D20026842F008020260026802F008020192A4
S31508001D30026842F040020260006800F0400001902C
S31508001D40086840F480200860086800F48020019044
S31508001D50802002900120039000240494059402A98F
S31508001D60114D2846FFF73AFE002228468021FFF744
S31508001D702CFF4FF4005002900394049402A90B48D8
S31508001D80FFF72CFE4FF44070029002200390049453
S31508001D90032005900720069002A90548FFF71EFEB6
S31508001DA007B030BD40380240000402400008024037
S31508001DB0000C0240F0B40D460D4B1B68C3F302231A
S31508001DC0C3F10704042C00D90424191D072901D2DC
S31508001DD0002300E0DB1E012606FA04F1491E29400D
S31508001DE099409E40761E16403143F0BC00F05CBD1B
S31508001DF00CED00E000F00701054A10684FF6FF03F6
S31508001E00184040EA01200349084310607047000063
S31508001E100CED00E00000FA05F8B51948016841F034
S31508001E2080510160006800F080500090154C2068D1
S31508001E3040F480302060FFF7CFFE05464FF47A76EF
S31508001E4006E0FFF7C9FE401BB04201D90320F8BDE2
S31508001E506068C003F5D5206840F400302060FFF7BD
S31508001E60BBFE054606E0FFF7B7FE401BB04201D9A8
S31508001E700320F8BD60688003F5D50020F8BD000092
S31508001E8040380240007000402DE9F04704460D46F0
S31508001E90002C17D0DFF83081D8F8000000F00F00CA
S31508001EA0A84211D2D8F8000020F00F002843C8F83D
S31508001EB00000D8F8000000F00F00A84204D0012066
S31508001EC0BDE8F0870120FBE72068404E810712D560
S31508001ED0400703D5306840F4E050306020780007AA
S31508001EE003D5306840F4604030603068A16820F05F
S31508001EF0F000084330602078C0072ED03349606868
S31508001F000839012806D0022809D0096889070BD4A0
S31508001F100120D5E70968890306D40120D0E70968B6
S31508001F20890101D40120CBE7316821F0030101437F
S31508001F303160FFF751FE074641F2883906E0FFF7A0
S31508001F404BFEC01B484501D90320B9E730686168D4
S31508001F5000F00C00B0EB810FF1D1D8F8000000F0CA
S31508001F600F00A8420ED9D8F8000020F00F00284329
S31508001F70C8F80000D8F8000000F00F00A84201D009
S31508001F8001209DE72078400705D53068E16820F4F0
S31508001F90E050084330602078000706D5306821698C
S31508001FA020F4604040EAC100306000F01BF8316858
S31508001FB0074AC1F30311515CC8400649086000206E
S31508001FC0FFF718FE00207BE7003C02400838024075
S31508001FD04A4900085400002001480068704700007C
S31508001FE05400002010B51748006810F00C01164878
S31508001FF016D04310042912D0082911D1114C241FD8
S31508002000216801F03F02216849020AD52068C0F319
S315080020108810A0FB03010023FEF75EF909E01846C5
S3150800202010BD21680023C1F38811A1FB0001FEF74A
S3150800203053F92168C1F30141491C4900B0FBF1F08D
S3150800204010BD0000083802400024F4002DE9F84FBE
S3150800205004464FF00008002C15D02078DFF8C0930E
S31508002060A9F10407C007A7F1040560D0D9F8000054
S31508002070C0F3810001280CD0D9F80000C0F3810014
S31508002080022803D00CE00120BDE8F88F386840022A
S3150800209006D5286880034AD5606870BB0120F3E737
S315080020A06068B0F5803F11D0A8B1B0F5A02F1BD05D
S315080020B0286820F480302860286820F4802028606A
S315080020C0606830B3FFF788FD06461EE0286840F4CE
S315080020D080302860F4E7286820F480302860286873
S315080020E020F480202860EBE7286840F480202860E8
S315080020F0286840F480302860E2E718E0FFF76CFDB6
S31508002100801B642801D90320BEE728688003F5D51B
S315080021100DE0FFF761FD064606E0FFF75DFD801B53
S31508002120642801D90320AFE728688003F5D420780E
S3150800213080074BD5D9F8000010F00C0F08D0D9F855
S315080021400000C0F38100022812D1386840020FD47B
S315080021502868800704D5E068012801D0012093E7A4
S315080021602868216920F0F80040EAC10028602DE0BF
S31508002170E068C8B1286840F001002860FFF72CFD28
S31508002180064606E0FFF728FD801B022801D9032032
S315080021907AE728688007F5D52868216920F0F800CD
S315080021A040EAC100286011E0286820F00100286094
S315080021B0FFF712FD064606E0FFF70EFD801B022814
S315080021C001D9032060E728688007F5D4207800073E
S315080021D030D5DFF84CA260690AF16C0AA8B1DAF8C2
S315080021E0000040F00100CAF80000FFF7F5FC0646BB
S315080021F006E0FFF7F1FC801B022801D9032043E71C
S31508002200DAF800008007F4D514E0DAF8000020F0C8
S315080022100100CAF80000FFF7DFFC064606E0FFF7F4
S31508002220DBFC801B022801D903202DE7DAF8000021
S315080022308007F4D42078400775D5DFF8E4A10AF1C1
S31508002240380ADAF80000C0000CD4DAF8000040F0CA
S315080022508050CAF80000DAF8000000F080500090BC
S315080022604FF00108DFF8BCB1DBF80000C00514D454
S31508002270DBF8000040F48070CBF80000FFF7ACFCF8
S31508002280064606E0FFF7A8FC801B642801D9032050
S31508002290FAE6DBF80000C005F4D5DFF884B1A068DB
S315080022A00BF1680B012814D0D0B1052825D0DBF82E
S315080022B0000020F00100CBF80000DBF8000020F059
S315080022C00400CBF80000A06870B3FFF785FC06464B
S315080022D02BE0DBF8000040F00100CBF80000F2E745
S315080022E0DBF8000020F00100CBF80000DBF8000066
S315080022F020F00400CBF80000E5E7DBF8000040F02A
S315080023000400CBF80000DBF8000040F00100CBF831
S315080023100000D8E7FFF760FC811B41F28830814254
S3150800232003D90320B0E61FE004E0DBF800008007CD
S31508002330F0D510E0FFF750FC064608E0FFF74CFC26
S31508002340811B41F28830814201D903209CE6DBF8E3
S3150800235000008007F2D4B8F1010F05D1DAF80000C1
S3150800236020F08050CAF80000A069E8B3D9F8001038
S31508002370C1F38101022951D0022807D0286820F02C
S3150800238080702860FFF728FC044642E0286820F0A1
S3150800239080702860FFF720FC064606E0FFF71CFC65
S315080023A0801B022801D903206EE628688001F5D42F
S315080023B054F81C0F4FF0FF336168E2680843A168C0
S315080023C003EB5202890141EA02410843217C40EAB3
S315080023D00160217D40EA01703860286840F080700D
S315080023E02860FFF7F9FB00E016E0044606E0FFF771
S315080023F0F3FB001B022801D9032045E62868800163
S31508002400F5D509E0FFF7E8FB001B022801D90320F0
S315080024103AE628688001F5D4002035E6012033E63F
S31508002420083802400070004010B5401EB0F1807FA9
S3150800243001D3012010BD4FF0E02460610F21601721
S3150800244000F032FA0020A06107202061002010BDAC
S3150800245010B5FFF7C3FBBDE8104000F07FBC0000D5
S3150800246070B50024494EC0284FF4004509D0B0F590
S31508002470407F27D0B0F5405F45D0B0F5404F63D0D8
S3150800248081E000F08BF8A0F5400040380BD04028DA
S315080024900DD0802811D000F0BBFB00F08FFB00F0B8
S315080024A09BFB04466FE000F0B3FB04466BE000F0CC
S315080024B01DF9002867D0344665E000F01FF908B317
S315080024C02C4660E000F06AF8314940180DD0B0F5A6
S315080024D0807F0ED0B0F5007F10D000F099FB00F099
S315080024E06DFB00F079FB04464DE000F091FB0446D5
S315080024F049E000F0FBF828B1344644E000F0FEF865
S3150800250000B12C463FE000F049F8224940180DD0AA
S31508002510B0F5805F0ED0B0F5005F10D000F078FB04
S3150800252000F04CFB00F058FB04462CE000F070FB72
S31508002530044628E000F0DAF828B3344623E000F031
S31508002540DDF800B32C461EE000F028F812494018C2
S3150800255009D0B0F5804F0AD0A8420DD100F0CEF8C8
S3150800256088B12C460FE000F053FB04460BE000F060
S31508002570BDF840B1344606E000F04AFB00F01EFB09
S3150800258000F02AFB0446204670BD00000024F40033
S3150800259000FFFFFC00F0FFCF00C0FF3F02490968BB
S315080025A0014041EA004070479038024070B5002467
S315080025B0484D03284FF4004607D00C2825D0B0F51F
S315080025C0406F42D0302861D071E000F087F86FF490
S315080025D0403140180BD001280DD0022810D000F049
S315080025E017FB00F0EBFA00F005FB04465FE000F08D
S315080025F00FFB04465BE000F079F800B32C4656E082
S3150800260000F07CF8D8B1344651E000F067F8A0F540
S315080026104020001F0BD004280DD0082810D000F049
S31508002620F7FA00F0CBFA00F0D7FA04463FE000F0DC
S31508002630EFFA04463BE000F059F800B12C4636E0C4
S3150800264000F05CF808B3344631E000F047F8224958
S3150800265040180DD0B0F5806F0ED0B0F5006F10D0D1
S3150800266000F0D6FA00F0AAFA00F0C4FA04461EE012
S3150800267000F0CEFA04461AE000F038F828B12C46E5
S3150800268015E000F03BF800B1344610E000F026F8FB
S31508002690A0F5401010380CD010280ED0202812D0E3
S315080026A000F0B6FA00F08AFA00F096FA04462046D8
S315080026B070BD00F0ADFA0446F9E700F017F80028F7
S315080026C0F5D02C46F3E700F019F80028EFD0344689
S315080026D0EDE700000024F40000FCFFF30249096856
S315080026E0014041EA004070479038024002480068BD
S315080026F0C0F34000704700000038024002480068F6
S31508002700C0F3400070470000703802400248006875
S3150800271000F03F0070470000043802400248006895
S3150800272000F48000704700000438024070B5044683
S315080027300D46002600202168C1F30001002960D15A
S31508002740EA686968AB6911432A691A431143226822
S31508002750344B1A4011432160A968626822F440523A
S315080027600A4362606969A26822F440720A43A26059
S315080027702D498C4203D10320FFF718FF33E02B497C
S315080027808C4203D10C20FFF711FF2CE028498C421C
S3150800279003D13020FFF70AFF25E026498C4204D1F1
S315080027A04FF44060FFF702FF1DE023498C4203D136
S315080027B0C020FFF755FE16E020498C4204D14FF49D
S315080027C04070FFF74DFE0EE01D498C4204D14FF4D0
S315080027D04050FFF745FE06E01A498C4203D14FF4F4
S315080027E04040FFF73DFE60B1296851B10126AA694C
S315080027F0B2F5004F07D000EB5100B0FBF1F080B204
S31508002800E060304670BD400000EB5100B0FBF1F0CF
S3150800281080B24FF6F0710140C0F342000143E16017
S31508002820EFE70000F369FFEF0010014000440040A5
S315080028300048004000140140004C00400050004091
S3150800284000780040007C0040002202488021FFF703
S31508002850BCB90000000402400149488070470000E6
S315080028605800002010B500F0F7FA0D4C6168884250
S315080028700DD321780B4859B10021217000228021FF
S31508002880FFF7A3F900F0E8FA61880844606010BD14
S315080028900121217001228021FFF797F9F2E7000054
S315080028A058000020000402400907090E002806DA2D
S315080028B000F00F0000F1E02080F8141D704700F1C9
S315080028C0E02080F8001470472DE9F0412348046899
S315080028D01C34234E4FF001074FF0000530784106AF
S315080028E007D52C3444F82C7CA583A577E577BDE875
S315080028F0F081C10701D084F84B50400708D594F8F9
S315080029004B00012804D1B4F84810201D01F098FFA7
S31508002910307800070DD594F84A00012809D184F8C3
S315080029204A50B4F8481021B184F84B70201D01F0C4
S3150800293087FF30788007DAD50A480188091F4029B9
S31508002940D5DC94F84B000028D1D107480068C9B2F5
S31508002950BDE8F041001D00F0C3BC0000B400002033
S31508002960980000209C000020AC00002004480021AC
S3150800297041700078002801D100F004B870470000C3
S315080029807000002038B51E4C6078002836D100F05B
S3150800299029FF00F061FA00F5FA70606000F05CFA51
S315080029A042F210752844A06001F036FA0021154A53
S315080029B011805180144801804180ADF80010ADF8AF
S315080029C002101248018041804EF6030001F066FAB3
S315080029D000F042FF04F10C0000F0F4FE062104F1B9
S315080029E00C0000F0A5FD00F0BDFDFDF73BFEA8427A
S315080029F002D22846FDF754FE0120207038BD00009B
S31508002A0070000020A8000020C8000020C400002094
S31508002A1010B504480078012801D100F005F8002017
S31508002A2010BD0000700000202DE9F05F00F028FFBF
S31508002A30404D002608B328804FF4006000F0A6FE3B
S31508002A403D4CA18988420AD1012001F03DFA288827
S31508002A5098B101F0ADF800F037FF2E800DE040F692
S31508002A60060000F093FEA189884206D101F04AF8D3
S31508002A70288810B100F028FF2E8000F0EDF92F4FBE
S31508002A80DFF8BC80DFF8BC90796888422ED301F560
S31508002A90FA717960002404EB840000EBC40008EBAB
S31508002AA0C000C9F80000022001F00EFA288820B1FB
S31508002AB001F07EF800F008FF2E80641C002CEAD096
S31508002AC00024DFF884A0DFF884B00AEB8410CBF882
S31508002AD00000052001F0F8F9288820B101F068F80F
S31508002AE000F0F2FE2E80641C002CEED000F0B4F943
S31508002AF0B968884205D342F210700844B86001F0FC
S31508002B0005F9002404EB840000EBC40008EBC000C0
S31508002B10C9F80000032001F0D7F9288820B101F090
S31508002B2047F800F0D1FE2E80641C002CEAD0BDE8E0
S31508002B30F09F00009C000020E43600207000002072
S31508002B40283D0020B4000020903D0020B800002059
S31508002B5030B50E4A1278012A16D10D4A13681C336D
S31508002B601A685A60002204E09D18845C2C72521C74
S31508002B7092B28A42F8D3091DA3F84810012083F8B7
S31508002B804A001868401C186030BD0000700000201C
S31508002B90B400002010B5FEF729FA18B1BDE81040B8
S31508002BA0FEF7DEB8002010BDFEF7F6B8FEF764B9EA
S31508002BB0FEF766B9FEF7A2B9FEF7BAB9044909687D
S31508002BC001F0F001034A0909515CC840704700004A
S31508002BD0083802404A4900080449096801F4E051E6
S31508002BE0034A02EB91210978C84070470838024029
S31508002BF05A4900080449096801F46041034A02EB8E
S31508002C0051310978C8407047083802405A490008C7
S31508002C100748006800F00C010648002906D0042978
S31508002C2003D0082902D100F009B80348704700000C
S31508002C30083802400024F40000127A0010B5FFF7A5
S31508002C406DFD0C4C18B1B0F5800F00D16410FFF77C
S31508002C505DFDB4FBF0F108480268C2F388125143DF
S31508002C60006800F44030012202EB10404000B1FB3E
S31508002C70F0F010BD0024F400043802400B4A106836
S31508002C80C1B2C0F307231944C0F30743194401EB43
S31508002C901061002013181B79194489B2401C382882
S31508002CA0F8D3C843401C80B27047000000000020DB
S31508002CB010B500F029F800280DD108490648086023
S31508002CC0002000220B181A71401C3828FAD3BDE8D8
S31508002CD0104000F039B810BDA2E742CE000000202F
S31508002CE070B504460D46002600F00EF838B1382CAB
S31508002CF005D225B1034820440079287001263046BC
S31508002D0070BD00000000002010B5002405480649E3
S31508002D100068884203D100F009F800B10124204672
S31508002D2010BD000000000020A2E742CE10B5002426
S31508002D30FFF7A4FF0349898F884200D10124204662
S31508002D4010BD00000000002010B5FFF797FF0149ED
S31508002D50888710BD000000207047000010B594B0A9
S31508002D602348016841F080510160006800F08050F6
S31508002D7001902048016841F440410160006800F470
S31508002D8040400190012007900004089002240D9409
S31508002D9080010E9008200F904FF4D870109011946F
S31508002DA0129407A8FFF752F918B1952112A0FDF75A
S31508002DB03AFCFFF731F818B19D210FA0FDF733FC57
S31508002DC00F2002900394002004904FF4A050059021
S31508002DD04FF480500690072102A8FFF755F80028FF
S31508002DE003D0AC2104A0FDF71EFC14B010BD0000F2
S31508002DF040380240007000402E2E5C6D61696E2ED0
S31508002E00630000001048016841F4700101600F4832
S31508002E10016841F0010101600C4A00210832116085
S31508002E2002680B4B1A400260031D0A4A1A600268C0
S31508002E3022F48022026005480C30016058060249D7
S31508002E40803908607047000088ED00E000380240CD
S31508002E50FFFFF6FE1030002400B500F01DF801480B
S31508002E60006800BD8400002000B500F00FF84FF0A0
S31508002E70E02004494161002181610522026102487E
S31508002E80016000BDBF4B0300840000204FF0E02125
S31508002E9000200861704700004FF0E0200069C00379
S31508002EA003D502480168491C016070478400002068
S31508002EB010B588B04FF4614001900020029003904D
S31508002EC004900C2105910690079001A9044C204610
S31508002ED0FFF72CFC216841F00101216008B010BD04
S31508002EE0004800400549CA69C2F34012002A03D0C7
S31508002EF0496A017001207047002070470048004069
S31508002F002DE9F04180460F461B4C00251B4E607884
S31508002F10002810D020783044401CFFF7E3FF012832
S31508002F2019D0FFF799FF61686431884200D9657046
S31508002F300020BDE8F0811148FFF7D4FF0128F7D13A
S31508002F403078401E3F28F3D8FFF786FF606025706B
S31508002F5001206070ECE72078401CC2B222703078FD
S31508002F6031469042E4D1491C4046FDF750FC657055
S31508002F70207838700120DCE7880000206C360020B5
S31508002F8070B5094DA862FFF767FF00F10A0405E06E
S31508002F90FDF733FCFFF760FFA04204D8E869C0F3E9
S31508002FA0C0100028F4D070BD0048004070B5054632
S31508002FB00E46402E03D9812108A0FDF734FB304682
S31508002FC0FFF7DEFF002406E0FDF717FC285DFFF794
S31508002FD0D7FF641CA4B2B442F6D370BD2E2E5C2E65
S31508002FE02E5C2E2E5C2E2E5C536F757263655C41CB
S31508002FF0524D434D375F53544D333246375C7561F6
S3150800300072742E630000000010B5084CFF21E170B1
S31508003010E21D4168A06C00F037F92071002060714C
S31508003020A0710820A4F8440010BD00001832002042
S3150800303070B500F0C9F90E4C01252570FF20E07027
S315080030400020102121716071FDF758FBA071FDF772
S315080030506BFBE071FDF768FB000A20726572A572CA
S315080030600820A4F84400BDE87040FFF7A1BD0000A1
S315080030701832002010B5054C0020207000F0A4F985
S31508003080FF20E0700120A4F8440010BD183200208B
S315080030900748FF21C1700749816400210171417108
S315080030A081710721C0F807100821A0F8441070475D
S315080030B018320020624900080648FF21C170002125
S315080030C00171427842718171C17101720621A0F8BD
S315080030D0441070471832002070B50446FDF70EFB01
S315080030E06178801E884204DABDE87040222000F02C
S315080030F071B9104DFF20E8700120A5F844006178E9
S3150800310049B1A86CA21CFFF757FD68B16178A86C95
S315080031100844A86470BDFFF73DFD0028FAD1BDE854
S315080031207040312000F056B9BDE87040312000F0FB
S3150800313051B900001832002010B5084C4168A06C3F
S31508003140FFF732FD28B1FF20E0700120A4F8440003
S3150800315010BDBDE81040312000F03CB918320020FF
S3150800316070B50546FDF7CAFA0B4C411E6A1CA06CE1
S31508003170FFF722FD58B1FF20E070FDF7BFFAA16CFA
S31508003180401E0844A0640120A4F8440070BDBDE8B0
S315080031907040312000F01EB918320020312000F0AE
S315080031A019B9000010B5FDF741FB0348FF21C170AE
S315080031B00121A0F8441010BD1832002070B5084C43
S315080031C0FF20E070002525716571FDF797FAA0715B
S315080031D0E571257265720720A4F8440070BD0000E9
S315080031E0183200200449FF22CA704068886401200A
S315080031F0A1F84400704700001832002070B5044654
S31508003200FDF77CFA6178401E884204DABDE8704012
S31508003210222000F0DFB8094D6168A9646278281D8C
S31508003220FDF7F5FAFF20E8706178A86C0844A864F1
S315080032306078401CA5F8440070BD000018320020D4
S31508003240002000F0C7B8000070B50546FDF756FA2D
S315080032506A78401E904204DABDE87040222000F0E9
S31508003260B9B8084C201DA16CFDF7D1FAFF20E07013
S315080032706978A06C0844A0646878401CA4F84400E7
S3150800328070BD0000183200202DE9F04104460E46B4
S315080032901746002505E014F8010B2844C5B2FDF7CA
S315080032A0ACFA761E701CF6D13D600120BDE8F081AF
S315080032B0054800210170816480F84310A0F8441085
S315080032C0817041707047000018320020034800786A
S315080032D0002801D0012070470020704718320020CE
S315080032E010B50178334CFF290FD02278012A60D116
S315080032F0F42921D013DCD02936D009DCC92930D0ED
S31508003300CC293DD0CF293ED137E0FFF791FE3DE0ED
S31508003310D1292FD0D2292AD0F32934D112E0F53970
S315080033200A2930D2DFE801F0050B2F2F2F112F14B1
S31508003330171AFFF789FF29E0FFF760FF26E0FFF776
S3150800334051FF23E0FFF760FE20E0FFF7A1FE1DE036
S31508003350FFF776FF1AE0FFF7AFFE17E0FFF78AFEE2
S3150800336014E0FFF7FDFE11E0FFF7B6FE0EE0FFF7EB
S3150800337025FF0BE0FFF7E0FE08E0FFF713FF05E087
S31508003380FFF70CFF02E0202000F024F894F8430031
S31508003390012802D1102000F01DF8B4F944100029C4
S315080033A007DD012284F84320E01CBDE8104000F048
S315080033B01BB810BD183200200249002081F84300CE
S315080033C070470000183200200149002048707047F5
S315080033D0183200200349FE22CA7008710220A1F89B
S315080033E0440070471832002089B2FDF7E9B9FF2179
S315080033F000F8011B70473522027001224270817065
S31508003400C01C704732210170042141700249496A83
S31508003410C0F80210801D7047B036002037210170B1
S315080034200321417001228270C17006210171401D7D
S315080034307047000036210170042141700249C969AC
S31508003440C0F80210801D7047B036002010B58B18E2
S315080034505B1E0BE00C784A7802EB042292B2104409
S3150800346080B2904201D2401C80B2891C9942F1D3A5
S31508003470994207D109780902084480B2884201D2E4
S31508003480401C80B210BDFFF7E7BC00002DE9F041F3
S315080034900446012020706070164D287EA07000201A
S315080034A0E070154E31686160208180216181134981
S315080034B00968E16020616061A06104F11C00D5E93A
S315080034C005120746FCF7ABFFA869C0F1100138449E
S315080034D0FCF7F2FF402104F12C00FCF7EDFF8021F8
S315080034E004F16C00FCF7E8FF7068C4F8EC00BDE86E
S315080034F0F0810000B0360020F0490008A80000203E
S3150800350000F03AB80749828C0A80C28C4A8006497C
S31508003510028D0A80428D4A800449028E0A80408EB6
S3150800352048807047A8000020C8000020C40000207A
S3150800353038B50B4C6061A1610025A5704FF6FF7088
S31508003540ADF80000ADF802004FF48641684601F078
S315080035508BF9606010B14FF488418180258038BDB1
S31508003560B0360020002102480180418070470000E3
S31508003570A8000020704700002DE9F84F0120814C73
S31508003580814D00264FF493784FF002094FF47A776D
S315080035904FF0030A218804F1080242F2107B0092D8
S315080035A041454FD009DCB1B1A1F580710F391FD063
S315080035B0012921D016290AD141E0A1F58071553992
S315080035C07DD001297CD015297BD016297AD0268072
S315080035D00220BDE8F88F0120A070276100F00AFAE2
S315080035E02169009800F045FA002040F20F11218069
S315080035F0F0B34FF4887020802878800703D40098A9
S3150800360000F02AFAA8B32878800703D500F092F9C3
S31508003610022836D020694EF66021884201DA400039
S315080036202061A0780228D9D1276100F0FBF9216929
S31508003630009800F01EFA002040F22511218018B3E8
S31508003640A4F800802878800703D4009800F004FACC
S31508003650E0B12878800703D500F06CF9052817D063
S315080036602069584537DC00F57A702061A07801E0BA
S3150800367003E004E00328D8D10CE00320A9E70020E2
S31508003680A7E784F80290CFE70320A2E70020A0E787
S3150800369084F802A03B48FFF735FF208C00F076F847
S315080036A04FEA0048608C00F071F840EA08004008CC
S315080036B04FF0004200EB4001C1EBC01103E018E0F7
S315080036C01BE02FE032E0B2EBC10F07D94FF47A7155
S315080036D04843206105E0268000207AE76FF0004025
S315080036E020612169009800F0C4F9002040F25511C4
S315080036F0218098B34FF4AB702080009800F0ACF9A5
S3150800370068B384F802902761FFF72CFFFFF732FFB2
S3150800371000F088F92169009800F0ABF900204FF411
S31508003720B571218000B340F26B102080287880079D
S3150800373003D4009800F090F9C0B12878800703D523
S3150800374000F0F8F8052813D02069584516DC00F56E
S315080037507A702061A0780328DAD10BE000E001E056
S31508003760032036E7002034E7032032E7002030E75D
S3150800377084F802A00348FFF7C5FE8EE726800020DE
S3150800378027E70000B036002098000020010241EA31
S31508003790102080B2704708B500200090FEF758FE4A
S315080037A0FFF786FAFCF782FF00206946FFF798FACA
S315080037B09DF80000012801D1FCF792FFFCF785FF70
S315080037C0FCE7000006490A7802704A7842708A784F
S315080037D08270CA78C2700A79027149794171704754
S315080037E04C00002010B517480821017000224270CD
S315080037F0272181706921C1705B21017145214171C1
S315080038001249114B0B6001234B600A8248618A6199
S31508003810CA61D80508620846FDF7ECFC0B49042383
S315080038200B4A0A48C831FDF768FC0A4A04230748C8
S31508003830A2F58071FDF72AFCBDE810400348FDF7A4
S315080038408ABE00004C00002000800240F0000020E4
S31508003850081A0020380200200748084902780A702A
S3150800386042784A7082788A70C278CA7002790A7178
S3150800387040794871704700004C00002090000020F5
S3150800388070B500250E48FDF775FCB8B90C4CA08F2D
S3150800389085B2216C0B482A46FCF7C1FD216B0868E6
S315080038A040F0004008600020A063216801F58051BF
S315080038B04A69120602D580224A618860284670BD88
S315080038C0F0000020E43600202DE9F0410126164FCD
S315080038D0FD6AFFF7C1FA00F1FA0407E0FCF78DFF6D
S315080038E0FFF7BAFAA04201D9002602E028680028A4
S315080038F0F4DB012E0BD10D480488F86A806822464D
S315080039000B49FCF78CFD08482146FDF746FE38684A
S3150800391000F580504169890603D5202141610021BF
S315080039204160BDE8F0810000F00000209C00002006
S31508003930E436002070B50F480468207802280DD1B7
S315080039400D490422201DFCF73EFD38B90B4D04F144
S315080039501C00D5E90512FCF736FD08B1002070BD3C
S31508003960206968620648018804F1F000BDE87040E5
S3150800397000F008B8AC000020F0490008B036002076
S315080039809C00002010B544180023194A29E0017844
S31508003990332920D006DC01290BD003290DD00629AE
S315080039A01CD10EE0352910D0362910D0FF2915D1A3
S315080039B01BE0D0F80210916210E0D0F802101163F3
S315080039C00CE0D0F80210D16208E0837806E0D0F85F
S315080039D00210D16102E0D0F8021011624178801C11
S315080039E00844A042D3D3184610BD184610BD00009F
S315080039F0B036002070B50A4D2C682046FFF746FD04
S31508003A00012104F1F000FFF7F6FCFFF707FDFFF7C9
S31508003A10EEFC01462868BDE87040091A00F010BFA0
S31508003A20AC00002070B50B4D2C682046FFF72EFD24
S31508003A30032104F1F000FFF7DEFCFFF7FBFCFFF7BC
S31508003A40E1FCFFF7D4FC01462868BDE87040091A76
S31508003A5000F0F6BEAC00002010B50446FFF713FDD3
S31508003A602168401A6168884201DB012010BD0020E8
S31508003A7010BD10B504466160FFF705FD206010BD56
S31508003A8030B5144DC2780A44D4B2EC70827802EB91
S31508003A901122D2B2AA7043786B7000782870B2EB04
S31508003AA0112F05D25B1CDBB26B700BB9401C28705A
S31508003AB0C8B284420DD2521CD0B2A870002808D1D0
S31508003AC06878401CC0B26870002802D12878401C6B
S31508003AD0287030BDC000002010B5094C0146E069C9
S31508003AE00830FFF7CDFFE06904F128010A78027271
S31508003AF04A7842728A788272C978C17210BD00000B
S31508003B00980000202DE9F047254D002029882A290C
S31508003B1002D22880BDE8F08728804FF40076214C31
S31508003B20214F224602F11601B4F81490881DB2F806
S31508003B3026C0B7F80080B9F5807F128D7B8809D03A
S31508003B40B145E7D1C445E5D19A42E3D1BDE8F0478E
S31508003B5000F0FEB8C445DDD19A42DBD100F0F8F892
S31508003B60A682D4F816002062618BA1840F4B1A68CE
S31508003B70C4F816209B886383C4F8062063812060F6
S31508003B80A180A08BE084E08B20853888A083788884
S31508003B90E0834FF4C160A0812A202880BAE700009C
S31508003BA09C000020E4360020A80000209000002099
S31508003BB02DE9F05FDFF82CA14FF6FF724A4B50460D
S31508003BC0BAF81E10008C9C8891421D6809D1904253
S31508003BD007D146480168CAF800108088AAF8040088
S31508003BE03FE0434B434F1A88B7F80090B7F8028076
S31508003BF001EA0206404F09EA0202964206D15A88AD
S31508003C0000EA020308EA0202934205D03B4801880B
S31508003C1039804088788001E0398078804FF0000B41
S31508003C20354B1B1F83F800B03E88DFF8D4C07F8869
S31508003C30197801EB41000CEB80000288964202D10C
S31508003C404288974204D0491CC9B219700829EFD393
S31508003C501978082912D04168CAF800100089AAF80C
S31508003C600400CAF80650AAF80A400820AAF80C0068
S31508003C70244801880E310180BDE8F09F1948FF22CB
S31508003C800621FCF711FCCAF820B0AAF824B0CAF835
S31508003C900650AAF80A40CAF81650AAF81A40AAF80E
S31508003CA02660AAF82870AAF81C90AAF81E804FF475
S31508003CB08070AAF81400AAF80E000820AAF81000C6
S31508003CC006208AF8120004208AF813004FF4C1600F
S31508003CD0AAF80C000C490348363008602A2109481E
S31508003CE00180C9E7E436002090000020F849000862
S31508003CF0C8000020A8000020D0000020C400002032
S31508003D00D03D00209C000020AC000020F0B50E4AF3
S31508003D109078401CC5B29570002313700B4E11782D
S31508003D2001EB410006EB8000048847883C4304D039
S31508003D30847A2C1B782C00DB0360491CC8B21070EF
S31508003D400828ECD3F0BD0000CC000020D03D0020B0
S31508003D502DE9F0412E4F4FF0000C87F800C02D4E8C
S31508003D603B7803EB430206EB8202148884B155883C
S31508003D7075B1B0F80080A0450AD14488AC4207D195
S31508003D800868506088881081B8789072BDE8F0811C
S31508003D905B1CDAB23A70082AE2D387F800C03B788F
S31508003DA003EB430206EB820214880CB9548824B14B
S31508003DB05B1CDBB23B70082BF1D33B78082B1DD17B
S31508003DC087F803C087F801C087F800C0BC783A783E
S31508003DD002EB420306EB8303FD789B7AE31AAB42B8
S31508003DE001DDFB707A70521CD2B23A70082AEED303
S31508003DF07A783A7002EB420206EB8202006810609B
S31508003E000868506088881081B8789072BEE700000C
S31508003E10CC000020D03D002010B5164900224A707B
S31508003E2001F10803487823F81020401CC0B24870F6
S31508003E300028F7D04A70104B487800EB800404EB52
S31508003E40C00403EBC4046276401CC0B24870002864
S31508003E50F2D04FF4806088814A70074B68334878FF
S31508003E6003EB8014A280401CC0B248700028F6D02C
S31508003E7010BD000098000020283D002010B5064916
S31508003E8014220020FFF7E2FA18B1BDE81040FFF748
S31508003E907DBC4FF6FF7010BDF236002010B5094AFA
S31508003EA00021517002F10803517833F811402CB102
S31508003EB0491CC9B251700029F6D010BD517823F8B3
S31508003EC0110010BD980000202DE9F05FF94FFC693C
S31508003ED00026F94D042805F1360A77D0C7F814A04C
S31508003EE0C7F818A003284FF0010B4FF0100909D0A6
S31508003EF0022814D0052805F12A047BD0A87B45287A
S31508003F0043D185E0607E00F00F000328F8D1208AAF
S31508003F100028F5D108203870FEF7D6FCAAE3E54953
S31508003F202431C878401C10F0FF00C8700ED188787C
S31508003F30401C10F0FF00887008D14878401C10F02B
S31508003F40FF00487002D10878401C0870BE80FE80C9
S31508003F50607E072812D0052810D0002815D0218A9F
S31508003F60A9B3A07E411EA1760FD2E07E082824D0F0
S31508003F70617E02290AD0012908D009E0A07E401CEA
S31508003F80C0B2A0767828BBD16676ECE0052814D0B6
S31508003F90042800D9042003218140A176E07E401C34
S31508003FA0E076607E00F00F000928EED2DFE800F028
S31508003FB0DBFC1114FBDBFBDBFB006676802038702C
S31508003FC0FEF782FC142085F82F00D6E39EE008E071
S31508003FD010E085F82F60E8E104203870FEF774FCDD
S31508003FE066E300F00F000328CFD108203870FEF7EB
S31508003FF06BFC3FE3386A80880028C6D0FE617C6186
S31508004000BC61FE80BE8008203870FFF779FA7DE033
S31508004010297C687C00EB0120B9888842B5D8B8802D
S31508004020287D8006B1D1687D0028AED1A148103020
S315080040300188408801B928B1EA8B8A42A5D1298C22
S315080040408142A2D1FFF71AFF4FF6FF7840459CD16F
S31508004050E87D062804D011280FD0012895D115E04F
S3150800406000F0FEFB404590D1944CA8466A8C6B8BB9
S315080040702146B5F81CC0A88C9BE0B8881C38B880C7
S315080040808E486830386200F1400269E095F82200EF
S315080040900828A9D185F822604FF6F771A88C8842BE
S315080040A002D30930A88401E00830A884688BE88325
S315080040B0A88B28847F481030018869834088A883A4
S315080040C0B9E38188F1B3AB8C8B4247D1C18829B15A
S315080040D06B8C8B4202D0B1F58A4F3FD1018809B962
S315080040E043885BB1414502D14388434506D06B8B73
S315080040F08B4233D1A98B438899422FD1FE61022086
S3150800410038707C61BC61FE80FFF7FAF9F9880029EE
S3150800411029D001F11C00B880020A2A746874386A2A
S31508004120027AAA751122EA750831C1F3072242EA12
S315080041300121E9842E8581886984C188A9845D491D
S31508004140103100E00AE00A886A834988A983018851
S31508004150E98340882884C7F814A05CE340303862B5
S31508004160386A9042ADD33EE394F819A0BAF1000F2D
S315080041701ED0B4F804A050451AD1B4F806A052458A
S3150800418016D1B4F800A0534512D1B4F802A0D4450C
S315080041900ED1FC613E7098F82F0041077CD56676F3
S315080041A02020387001E031E2FDE0FEF78DFB1AE3CE
S315080041B068348C42D8D998F82F2002F03F02022A98
S315080041C010D1F8817E703B4B08337A7833F8124069
S315080041D0844202D100247E705FE0521CD2B27A700B
S315080041E0002AF2D098F82F004007BCD4142088F88B
S315080041F02F002820B880502088F82E0098F82930FB
S3150800420098F82D0088F8290098F8281098F82C00B6
S3150800421088F8280088F82C1098F8272098F82B009A
S3150800422088F8270088F82B2098F82600787098F8E0
S315080042302A4088F8264088F82A005B1C13F0FF03FA
S3150800424088F82D300ED1491C11F0FF0188F82C1082
S3150800425008D1521C12F0FF0188F82B1002D1401C1D
S3150800426088F82A00B8F82200F881B8F82410A8F8C7
S315080042702210A8F82400B8F81A00A8F81E00B8F802
S315080042801C00A8F820000B4810300188A8F81A105E
S315080042904088A8F81C00AFE2AEE07A7802EB82000C
S315080042A000EBC20001EBC000437E4BB1072B0FD0D9
S315080042B015E0000098000020E4360020283D002084
S315080042C0787800EB800202EBC00001EBC0040BE03B
S315080042D024B1837E94F81AC0634500D90446521C5B
S315080042E0D0B278700028D8D0002C71D0BA46FC61BC
S315080042F00320A0762076A6750420E075E676B8F841
S315080043002400A080B8F82200E080B8F81A002080BF
S31508004310B8F81C00608084F819B0F9480178217350
S31508004320417861738178A173C078E073A4F810B0FE
S3150800433098F82900E07298F82800A07298F82700E3
S31508004340607298F8260020720120FFF7C5FB98F8DE
S315080043502E0000F0F001502925D98AF801606FF087
S31508004360040101EB101319E008EB000292F836106D
S315080043708AF80210B9B1012902D0022904D007E04F
S31508004380401C8AF8010009E092F83710042920D069
S3150800439092F8371039B108448AF801009AF80100F2
S315080043A0B0EB830FE0DB85F82F902E35687840F068
S315080043B00200687002202872042068720620A8721B
S315080043C00A20E8722C20B880602005F82E09D9E169
S315080043D0FEE09AF8010092F83810404490F8390047
S315080043E040EA0120AAF80E0040F20A61884200D984
S315080043F008466082A082D6E798F82E100909890037
S315080044007970BA88511A143989B2B980627E02F075
S315080044100F02022A03D100F03F02122A17D009B967
S31508004420810714D098F826104346227A91427DD106
S3150800443093F82710627A9142F9D193F82810A27A54
S315080044409142F4D193F82910E27A9142EFD1C0064D
S31508004450C2463DD5218AD9B304F10C00FFF710FBFB
S31508004460A74B9AF82A101B1D1878814230D19AF862
S315080044702B20D64659788A422AD19EF82CC09A789B
S31508004480944525D19EF82DC0DB789C4520D1207314
S315080044906173A273E373E07EA8B9207EA17E401AF9
S315080044A0A17DA0EBD10040B20144C9B2A175002894
S315080044B001DA404240B2E27DA0EB92001044E0757A
S315080044C000EBD100207687F800B0207EA076268201
S315080044D0607E00F00F0109297AD2DFE801F079053C
S315080044E0177AF8F7F627F5003878C00770D0032052
S315080044F06076402038702682B88818B14221397013
S31508004500FFF7EAFAFE80FEF7DFF9B3E03878C0076E
S3150800451005D09AF82F0000F03F00122807D0202077
S315080045203870FEF7D1F9F86946765BE623E19AF822
S315080045302E0000F0F001502920D97E706FF004019A
S3150800454001EB101316E00AEB000292F83610B97068
S31508004550A1B1012902D0022903D006E0401C7870D7
S3150800456008E092F83710042921D092F8371029B1BB
S31508004570084478707878B0EB830FE4DB0320607624
S315080045809AF8260020729AF8270060729AF828008E
S31508004590A0729AF82900E0720120FFF79DFA4220DE
S315080045A038702682BE80FE80FEF78EF962E0787843
S315080045B092F83810504490F8390040EA0120F88102
S315080045C040F20A61884200D908466082A082D5E78F
S315080045D046E09AF82F10CA071CD0C2061AD4208AB9
S315080045E0F0BBB888401C80B2FFF776FA387840F0FE
S315080045F010003870B98811B140F002003870FEF723
S3150800460063F9A4F810B008206076E676112085F8DC
S315080046102F00B2E089060BD59AF834209AF835109F
S3150800462041EA02217A690A447A61BA88511AB9803C
S31508004630B98841B1C00606D4387840F0020038700F
S315080046400846FFF749FA9AF830109AF8310000EB55
S31508004650012080B2F881A18A814200D310B900E016
S315080046604DE0F981F88960823878800747D0FE8066
S31508004670FEF72AF93878810605D5FE806676142075
S3150800468085F82F0079E0C10609D5FE80A4F810B098
S3150800469004206076E676112085F82F006DE0F9880B
S315080046A029B1C00700D02682208A88B1F880E6762C
S315080046B0B8697861F88890B1208A80B12830B880C6
S315080046C0182085F82F005AE011E086E03EE019E050
S315080046D0608A884200D2F880F8882082E7E738782E
S315080046E080070CD52820B88085F82F9047E03878C1
S315080046F0C00778D0667687F80090FEF7E5F872E08E
S31508004700BC000020B88808B1FFF7E6F99AF82F0030
S31508004710C00711D03878C00704D007206076A6767F
S31508004720268201E0062060760120FFF7D5F987F892
S315080047300090FEF7C9F81EE03878C00703D00520B8
S31508004740607626824FE0B888A8B94CE0B88808B1E8
S31508004750FFF7C2F99AF82F00C0070AD0072060763B
S31508004760A6760120FFF7B8F987F80090FEF7ACF8AF
S3150800477001E0B88880B388F82F902820B8805020A8
S3150800478085F82E001835207AA874607AE874A07A1D
S315080047902875E07A6875207BA873607BE873A07B30
S315080047A02874E07B6874062005F8010CA1886981E5
S315080047B0E188A98121490A886A804988A9802188CF
S315080047C0E98061882981183D617EC9060FD585F87B
S315080047D0316085F830600FE005E03878C00702D010
S315080047E007206076A676BE803E70BDE8F09F85F805
S315080047F030000A2085F831004020A875B888010ADB
S315080048002974687485F8356085F834606E8600F01A
S3150800481027F8C04368864520A873EE736E752E7513
S315080048207889401C7881010AA974E8742E83FFF7F9
S3150800483025FBC04328833E70D7E70000A800002068
S315080048400346002908DD05488AB2C280806983428A
S3150800485002D01946FBF7E3BD704700009800002018
S31508004860062000F04DB800002DE9F04104460F4639
S31508004870214B0025214A4FF4FA484FF48056908977
S31508004880401C80B29081404500D39681557090892E
S31508004890FEF77CFF0146507803EB801CBCF804C089
S315080048A06145ECD0401CC0B250700028EFD0002003
S315080048B05570517803EB8116B688A6B1491CC9B262
S315080048C051700029F5D090B191890A0242EA112166
S315080048D08180C7806CB12188018061884180402130
S315080048E00172BDE8F081507803EB8010EBE70020F9
S315080048F0F7E70560F3E70000903D002098000020E8
S3150800490010B50E496FF013034A7C097C03EB0121AD
S3150800491011448CB2204480B2084908221A31FEF7A5
S3150800492095FD064922462231FEF790FD18B1BDE8ED
S315080049301040FEF72BBF4FF6FF7010BDE43600207F
S315080049404FF04070E1EE100A7047000000000000CA
S31508004950000001020304060708090000000001021E
S3150800496003044F70656E424C540000000080000836
S31508004970008000000100000000000108008000001F
S31508004980020000000080010800800000030000000B
S3150800499000000208000002000400000000000408ED
S315080049A000000400050000000000080800000400DC
S315080049B00600000000000C080000040007000000C4
S315080049C00000100800000400080000000000140899
S315080049D00000040009000000000018080000040098
S315080049E00A00000000001C08000004000B0000007C
S315080049F0ADDE122363825363FFFFFFFFFFFF000054
S31508004A00204A0008400000209400000034020008F4
S31508004A10B44A0008D4000020BC4300005002000835
S31508004A200100000010000000000000000000000067
S31508004A30000000000024F400000000000000000050
S31508004A400000000000000000000000000400000054
S31508004A500001000000000000000000000000000047
S31508004A600000000000000000000000000000000038
S31508004A700000000000000000000000000000000028
S31508004A800000000000000000000000000000000018
S31508004A900000000000000000000000000000000008
S31508004AA000000000000000000000000000000000F8
S30908004AB000000000F4
S705080001F9F8
